:0E0000000C947F000C9400000C9400000C94F3
:10000E0000000C9400000C9400000C9400000C9462
:10001E0000000C9400000C9400000C9400000C9452
:10002E0000000C9400000C9400000C9400000C9442
:10003E0000000C9400000C9400000C9400000C9432
:10004E0000000C9400000C9400000C9400000C9422
:10005E00BD000C9400000C9400000C9400000C9455
:10006E0000000C9400000C9400000C9400000C9402
:10007E0000000C9400000C9400000C9400000C94F2
:10008E0000000C9400000C9400000C9400000C94E2
:10009E0000000C9400000C9400000C9400000C94D2
:1000AE0000000C9400000C9400000C9400000C94C2
:1000BE0000000C9400000C9400000C9400000C94B2
:1000CE0000000C9400000C9400000C9400000C94A2
:1000DE0000000C9400003F065B4F666D7D277F6F1E
:1000EE0000000A00000AE40002000300EE00000017
:1000FE00F894EE27EFBBF1E0F5BFE5BFE093740097
:10010E00E0937500F8E1A895A4B7A77FA4BFF0937C
:10011E006000E09360008DE0A2E0BB27ED938A952E
:10012E00E9F780E090E2A0E0B2E0ED930197E9F705
:10013E00E0EFF0E085919591009761F0A591B59172
:10014E0005901590BF01F00105900D920197E1F712
:10015E00FB01F0CF8BBF8CBFE0E0EEBBEFEFEDBF4E
:10016E00E1E2EEBFC0E0DAE00C943801AA93BA9354
:10017E00EA93FA93EFB7EA93ABE0BAE0ED91FD9113
:10018E003196FE93EE93A0910B0AB0910C0AA43611
:10019E00E0E0BE0781F4E1E0F0E03E0E4F1EE0E04D
:1001AE00E0930B0AE0930C0AEFE0F7E2E315F40597
:1001BE0011F433244424E6B5EA5FE6BDE991EFBFBE
:1001CE00F991E991B991A99118952297E0E0E88308
:1001DE00E9830E947901A885B985E8EEF3E00E94D3
:1001EE006301EE83FF83A885B985E8EEF3E00E94F4
:1001FE007601DF01E4E6F0E00E946301AF01A8851D
:10020E00B985E4E6F0E00E947601DF01EAE0F0E075
:10021E000E9463018F01A885B985EAE0F0E00E9493
:10022E0076019F01EEE0E0930801EE81FF81E05040
:10023E00F64FE08129D0EDE02ED0A40FB51FEC9142
:10024E0023D0EBE028D0A00FB11FEC911DD0E7E03A
:10025E0022D0A20FB31FEC9117D00E9480012A96D4
:10026E000895EFEFE1B9E0930701E0E0E4BDE3E0CC
:10027E00E5BDE6E0E6BDE1E0E0936E0078944A92DB
:10028E003A92A3DFFCCFFFCFE2B9E5E0F0E0FA93BC
:10029E00EA930C945701E0930801A0E0BAE00895A8
:1002AE00E991F991309639F080EA9FE00197F1F7E4
:1002BE00A8953197C9F708950024112490E1AA0F4B
:1002CE00BB1F001C111C0E1A1F0A18F40E0E1F1E47
:1002DE0001C0A1609A9599F7FD01D0010895ECDF58
:1002EE00FD0108955A934A933A932A931A930A93C7
:1002FE0008955D814C813B812A8119810881089581
:00000001FF
